:020000040000FA
:0408000030EF05F0E0
:1008100003B23DEF04F0F2B458EF04F09EB060EF85
:1008200004F09EB268EF04F0F2A81AEF04F0F2B2FE
:100830001CEF04F00EEF05F0CD90F29207BC078E8E
:10084000078C9EA029EF04F00101463F29EF04F038
:10085000472B07AE34EF04F0CECF51F1CFCF52F19A
:1008600046C153F147C154F1CF6ACE6A0101466BCC
:10087000476B9E90CD800EEF05F00392030103EECF
:1008800000F080517F0BE92604C0EFFF802B8151DF
:10089000805D700BD8A48B8200008051815D700B4D
:1008A000D8A48B9281518019D8B407900EEF05F02F
:1008B000F2940101383F0EEF05F0392B0EEF05F0F1
:1008C0009E900101463F0EEF05F0472B0EEF05F01D
:1008D0009E92C3CF48F1C4CF49F1C28207B492EFD0
:1008E00004F03AC13EF13BC13FF13CC140F13DC192
:1008F00041F151C155F152C156F153C157F154C1A3
:1009000058F1010148514E2749514F23E86A5023BD
:100910000D2E92EF04F04FC14AF150C14BF14E6BD6
:100920004F6B506B0201002F0EEF05F03C0E006F75
:1009300001015D67A3EF04F05E67A3EF04F05F675A
:10094000A3EF04F06067A7EF04F0D7EF04F061C1F4
:1009500000F162C101F163C102F164C103F101015F
:10096000010E046F000E056F000E066F000E076F7C
:10097000D1EC11F000C161F101C162F102C163F17A
:1009800003C164F10067CCEF04F00167CCEF04F021
:100990000267CCEF04F00367D7EF04F05DC161F1AB
:1009A0005EC162F15FC163F160C164F10E80D57E0A
:1009B000D5BE32D0D6CF3AF1D7CF3BF138C13CF1DA
:1009C000E86AE8CF3DF1010147A7F2EF04F0079C88
:1009D000079E0101000E516F600E526F3D0E536F66
:1009E000080E546F01013ABF02EF05F03B6702EFBA
:1009F00005F03C6702EF05F03D6702EF05F0F28875
:100A000007EF05F0F298516B526B536B546BD76A3A
:100A1000D66A0101386B396B0EEF05F002C0E0FFBA
:100A2000005001C0D8FF1000A6B214EF05F00CC0B2
:100A3000A9FF0BC0A8FFA69EA69CA684F29E550EF9
:100A4000A76EAA0EA76EA682F28EA694A6B226EF75
:100A500005F01200A96EA69EA69CA680A8501200C2
:100A6000076A0E6A0F010E0EC16E860EC06E030E6F
:100A7000C26E0F01896A110E926E080E8A6EF10E17
:100A8000936E8B6A800E946EF18E0D6A4E6B4F6B77
:100A9000506B4A6B4B6B0F01280ED56EF28AB00E6D
:100AA000CD6E9D800101516B526B536B546B556B36
:100AB000566B576B586B596B5A6B5B6B5C6B079C37
:100AC000079E760ECA6E9D8202013C0E006FCC6AB4
:100AD000160E2AEC05F0E8CF00F1170E2AEC05F00F
:100AE000E8CF01F1180E2AEC05F0E8CF02F1190E5B
:100AF0002AEC05F0E8CF03F1010103AF9AEF05F00E
:100B0000C8EC12F0160E0C6E00C10BF014EC05F0E0
:100B1000170E0C6E01C10BF014EC05F0180E0C6EE4
:100B200002C10BF014EC05F0190E0C6E03C10BF0B2
:100B300014EC05F000C15DF101C15EF102C15FF18D
:100B400003C160F100C161F101C162F102C163F151
:100B500003C164F11A0E2AEC05F0E8CF00F11B0E78
:100B60002AEC05F0E8CF01F11C0E2AEC05F0E8CFE5
:100B700002F11D0E2AEC05F0E8CF03F1010103AFED
:100B8000F0EF05F0C8EC12F01A0E0C6E00C10BF07D
:100B900014EC05F01B0E0C6E01C10BF014EC05F00B
:100BA0001C0E0C6E02C10BF014EC05F01D0E0C6E49
:100BB00003C10BF014EC05F01A0E2AEC05F0E8CF97
:100BC00000F11B0E2AEC05F0E8CF01F11C0E2AEC17
:100BD00005F0E8CF02F11D0E2AEC05F0E8CF03F195
:100BE00000C165F101C166F102C167F103C168F19D
:100BF000240EAC6E900EAB6E240EAC6E080EB86E6A
:100C0000000EB06E1F0EAF6E0401806B816B0F0182
:100C1000900EAB6E0F019D8A0301806B816BA26BFE
:100C20008B9207900001F28EF28C07B0DCEF0FF090
:100C30000EB099EF0AF00301805181197F0BD8B4EF
:100C4000DCEF0FF013EE00F081517F0BE126812BDA
:100C5000E7CFE8FFE00BD8B4DCEF0FF023EE82F033
:100C6000A2511F0BD926E7CFDFFFA22BDF50780A56
:100C7000D8A4DCEF0FF0078061C100F162C101F17F
:100C800063C102F164C103F10101040E046F000E9F
:100C9000056F000E066F000E076FD1EC11F000AF6C
:100CA0005BEF06F00101030E616F000E626F000E34
:100CB000636F000E646F03018251720AD8B499EF1A
:100CC0000AF08251520AD8B499EF0AF08251630AAD
:100CD000D8B49CEF0CF08251690AD8B46EEF08F0DA
:100CE00082517A0AD8B481EF09F08251490AD8B406
:100CF00085EF07F08251500AD8B4A3EF06F0825175
:100D0000700AD8B4E6EF06F08251540AD8B411EF55
:100D100007F08251740AD8B457EF07F0D1EF0CF006
:100D2000040114EE00F080517F0BE12682C4E7FF3E
:100D3000802B12000D0E826F90EC06F00A0E826F6F
:100D400090EC06F0120083C31EF184C31FF185C32B
:100D500020F186C321F187C322F188C323F189C31F
:100D600024F18AC325F18BC326F18CC327F101013D
:100D700015EC13F08DEC12F0160E0C6E00C10BF09A
:100D800014EC05F0170E0C6E01C10BF014EC05F01D
:100D9000180E0C6E02C10BF014EC05F0190E0C6E5F
:100DA00003C10BF014EC05F000C15DF101C15EF16F
:100DB00002C15FF103C160F100C161F101C162F1E3
:100DC00002C163F103C164F185EF07F083C31EF133
:100DD00084C31FF185C320F186C321F187C322F1AB
:100DE00088C323F189C324F18AC325F18BC326F17B
:100DF0008CC327F1010115EC13F08DEC12F000C14A
:100E00005DF101C15EF102C15FF103C160F100C19A
:100E100061F101C162F102C163F103C164F185EFC7
:100E200007F083C31EF184C31FF185C320F186C37D
:100E300021F187C322F188C323F189C324F18AC336
:100E400025F18CC326F18DC327F1010115EC13F0B8
:100E50008DEC12F00101000E046F000E056F010E03
:100E6000066F000E076FE0EC11F01A0E0C6E00C159
:100E70000BF014EC05F01B0E0C6E01C10BF014EC22
:100E800005F01C0E0C6E02C10BF014EC05F01D0EEB
:100E90000C6E03C10BF014EC05F000C165F101C14B
:100EA00066F102C167F103C168F185EF07F083C302
:100EB0001EF184C31FF185C320F186C321F187C3CE
:100EC00022F188C323F189C324F18AC325F18CC39D
:100ED00026F18DC327F1010115EC13F08DEC12F012
:100EE0000101000E046F000E056F010E066F000E6B
:100EF000076FE0EC11F000C165F101C166F102C1BC
:100F000067F103C168F185EF07F0160E2AEC05F0D2
:100F1000E8CF00F1170E2AEC05F0E8CF01F1180E2A
:100F20002AEC05F0E8CF02F1190E2AEC05F0E8CF23
:100F300003F16BEC12F01EC182F40401300E822723
:100F400090EC06F01FC182F40401300E822790EC71
:100F500006F020C182F40401300E822790EC06F0E6
:100F600021C182F40401300E822790EC06F022C1E8
:100F700082F40401300E822790EC06F023C182F443
:100F80000401300E822790EC06F024C182F40401A3
:100F9000300E822790EC06F025C182F40401300E59
:100FA000822790EC06F026C182F40401300E8227DD
:100FB00090EC06F027C182F40401300E822790ECF9
:100FC00006F00401730E826F90EC06F004012C0E03
:100FD000826F90EC06F05DC100F15EC101F15FC16E
:100FE00002F160C103F16BEC12F01EC182F4040146
:100FF000300E822790EC06F01FC182F40401300EFF
:10100000822790EC06F020C182F40401300E822782
:1010100090EC06F021C182F40401300E822790EC9E
:1010200006F022C182F40401300E822790EC06F013
:1010300023C182F40401300E822790EC06F024C113
:1010400082F40401300E822790EC06F025C182F470
:101050000401300E822790EC06F026C182F40401D0
:10106000300E822790EC06F027C182F40401300E86
:10107000822790EC06F00401730E826F90EC06F06C
:1010800004012C0E826F90EC06F01A0E2AEC05F08B
:10109000E8CF00F11B0E2AEC05F0E8CF01F11C0EA1
:1010A0002AEC05F0E8CF02F11D0E2AEC05F0E8CF9E
:1010B00003F1EBEC0CF004012C0E826F90EC06F0C7
:1010C00065C100F166C101F167C102F168C103F1B8
:1010D000EBEC0CF09AEC06F0D1EF0CF00401690E89
:1010E000826F90EC06F004012C0E826F90EC06F0FB
:1010F0000101040E006F000E016F000E026F000E62
:10110000036F6BEC12F020C182F40401300E8227D1
:1011100090EC06F021C182F40401300E822790EC9D
:1011200006F022C182F40401300E822790EC06F012
:1011300023C182F40401300E822790EC06F024C112
:1011400082F40401300E822790EC06F025C182F46F
:101150000401300E822790EC06F026C182F40401CF
:10116000300E822790EC06F027C182F40401300E85
:10117000822790EC06F004012C0E826F90EC06F0B2
:101180000101030E006F000E016F000E026F000ED2
:10119000036F6BEC12F020C182F40401300E822741
:1011A00090EC06F021C182F40401300E822790EC0D
:1011B00006F022C182F40401300E822790EC06F082
:1011C00023C182F40401300E822790EC06F024C182
:1011D00082F40401300E822790EC06F025C182F4DF
:1011E0000401300E822790EC06F026C182F404013F
:1011F000300E822790EC06F027C182F40401300EF5
:10120000822790EC06F004012C0E826F90EC06F021
:101210000101100E006F000E016F000E026F000E34
:10122000036F6BEC12F020C182F40401300E8227B0
:1012300090EC06F021C182F40401300E822790EC7C
:1012400006F022C182F40401300E822790EC06F0F1
:1012500023C182F40401300E822790EC06F024C1F1
:1012600082F40401300E822790EC06F025C182F44E
:101270000401300E822790EC06F026C182F40401AE
:10128000300E822790EC06F027C182F40401300E64
:10129000822790EC06F004012C0E826F90EC06F091
:1012A000200EF86EF76AF66A04010900F5CF82F4A1
:1012B00090EC06F00900F5CF82F490EC06F00900FE
:1012C000F5CF82F490EC06F00900F5CF82F490ECB3
:1012D00006F00900F5CF82F490EC06F00900F5CF96
:1012E00082F490EC06F00900F5CF82F490EC06F061
:1012F0000900F5CF82F490EC06F09AEC06F0D1EFFD
:101300000CF08351630AD8A4D1EF0CF08451610A28
:10131000D8A4D1EF0CF085516C0AD8A4D1EF0CF011
:101320008651410A42E08651440A1BE08651420A36
:10133000D8B4E8EF09F08651350AD8B45AEF0EF068
:101340008651360AD8B4AEEF0EF08651370AD8B4BB
:1013500016EF0FF08651380AD8B474EF0FF0D1EFC2
:101360000CF00798079A04017A0E826F90EC06F051
:101370000401780E826F90EC06F00401640E826F17
:1013800090EC06F081A8CCEF09F00401550E826FB5
:1013900090EC06F0D1EF09F004014C0E826F90EC56
:1013A00006F09AEC06F0D1EF0CF00788079A0401DA
:1013B0007A0E826F90EC06F00401410E826F90EC81
:1013C00006F00401610E826F90EC06F0C2EF09F0A6
:1013D0000798078A04017A0E826F90EC06F00401E8
:1013E000420E826F90EC06F00401610E826F90EC69
:1013F00006F0C2EF09F00101620E046F010E056FE5
:10140000000E066F000E076F59C100F15AC101F1BD
:101410005BC102F15CC103F1D1EC11F003BF58EFE5
:101420000AF00E0E2AEC05F0E8CF0CF10F0E2AECB4
:1014300005F0E8CF0DF1100E2AEC05F0E8CF0EF123
:10144000110E2AEC05F0E8CF0FF11AEC11F059C19A
:1014500004F15AC105F15BC106F15CC107F1D1ECA1
:1014600011F00782DEEC10F01AEC11F00792DEECBE
:1014700010F059C100F15AC101F15BC102F15CC128
:1014800003F10792DEEC10F0CC0E046FE00E056F56
:10149000870E066F050E076FD1EC11F000C10CF13D
:1014A00001C10DF102C10EF103C10FF190EF0AF07D
:1014B0000101800E006F1A0E016F060E026F000E02
:1014C000036F42C104F143C105F144C106F145C1B6
:1014D00007F1D1EC11F003AF71EF0AF0C8EC12F094
:1014E00012000E0E2AEC05F0E8CF0CF10F0E2AECDC
:1014F00005F0E8CF0DF1100E2AEC05F0E8CF0EF163
:10150000110E2AEC05F0E8CF0FF142C100F143C102
:1015100001F144C102F145C103F10782DEEC10F094
:101520000CC100F10DC101F10EC102F10FC103F1B7
:1015300012008251520A03E10E82A0EF0AF00E92CD
:10154000078455C159F156C15AF157C15BF158C1D1
:101550005CF13EC142F13FC143F140C144F141C1A0
:1015600045F14AC14CF14BC14DF107940EA0D7EFA4
:101570000AF001016567C4EF0AF06667C4EF0AF07C
:101580006767C4EF0AF06867C8EF0AF0D7EF0AF0A0
:10159000FBEC09F065C104F166C105F167C106F114
:1015A00068C107F1D1EC11F003BF99EF0CF0FBEC2F
:1015B00009F00101000E046F000E056F010E066FA9
:1015C000000E076FFFEC11F00401720E826F90ECB9
:1015D00006F004012C0E826F90EC06F06BEC12F01A
:1015E0001D67F8EF0AF00401200E826FFBEF0AF08E
:1015F00004012D0E826F90EC06F024C182F40401E8
:10160000300E822790EC06F025C182F40401300EE2
:10161000822790EC06F004012E0E826F90EC06F00B
:1016200026C182F40401300E822790EC06F027C117
:1016300082F40401300E822790EC06F004016D0E56
:10164000826F90EC06F004012C0E826F90EC06F095
:1016500042C100F143C101F144C102F145C103F1AE
:1016600001016BEC12F01EC182F40401300E8227DE
:1016700090EC06F01FC182F40401300E822790EC3A
:1016800006F020C182F40401300E822790EC06F0AF
:1016900021C182F40401300E822790EC06F022C1B1
:1016A00082F40401300E822790EC06F023C182F40C
:1016B0000401300E822790EC06F024C182F404016C
:1016C000300E822790EC06F025C182F40401300E22
:1016D000822790EC06F026C182F40401300E8227A6
:1016E00090EC06F027C182F40401300E822790ECC2
:1016F00006F00401480E826F90EC06F004017A0EA9
:10170000826F90EC06F004012C0E826F90EC06F0D4
:1017100059C100F15AC101F15BC102F15CC103F191
:1017200001016BEC12F01EC182F40401300E82271D
:1017300090EC06F01FC182F40401300E822790EC79
:1017400006F020C182F40401300E822790EC06F0EE
:1017500021C182F40401300E822790EC06F022C1F0
:1017600082F40401300E822790EC06F023C182F44B
:101770000401300E822790EC06F024C182F40401AB
:10178000300E822790EC06F025C182F40401300E61
:10179000822790EC06F026C182F40401300E8227E5
:1017A00090EC06F027C182F40401300E822790EC01
:1017B00006F00401630E826F90EC06F004012C0E1B
:1017C000826F90EC06F059C100F15AC101F15BC182
:1017D00002F15CC103F101010A0E046F000E056FF6
:1017E000000E066F000E076FE0EC11F0000E046FA4
:1017F000120E056F000E066F000E076FFFEC11F062
:101800006BEC12F01EC182F40401300E822790ECC2
:1018100006F01FC182F40401300E822790EC06F01E
:1018200020C182F40401300E822790EC06F021C121
:1018300082F40401300E822790EC06F022C182F47B
:101840000401300E822790EC06F023C182F40401DB
:10185000300E822790EC06F024C182F40401300E91
:10186000822790EC06F004012E0E826F90EC06F0B9
:1018700025C182F40401300E822790EC06F026C1C7
:1018800082F40401300E822790EC06F027C182F426
:101890000401300E822790EC06F00401730E826F73
:1018A00090EC06F004012C0E826F90EC06F0C8EC70
:1018B00012F04CC100F14DC101F1FAEC0DF00EB285
:1018C00065EF0CF00EA097EF0CF004012C0E826F68
:1018D00090EC06F0200EF86EF76AF66A0401090033
:1018E000F5CF82F490EC06F00900F5CF82F490EC8D
:1018F00006F00900F5CF82F490EC06F00900F5CF70
:1019000082F490EC06F00900F5CF82F490EC06F03A
:101910000900F5CF82F490EC06F00900F5CF82F4CF
:1019200090EC06F00900F5CF82F490EC06F09AEC0A
:1019300006F00E90D1EF0CF00401630E826F90EC74
:1019400006F004012C0E826F90EC06F0D6EC0CF041
:1019500004012C0E826F90EC06F049EC0DF00401AE
:101960002C0E826F90EC06F0C5EC0DF004012C0EED
:10197000826F90EC06F00101F80E006FCD0E016F42
:10198000660E026F030E036FEBEC0CF004012C0EDD
:10199000826F90EC06F0DBEC0DF09AEC06F0D1EFE4
:1019A0000CF00301A26B0790DCEF0FF0D8900E0E45
:1019B0002AEC05F0E8CF00F10F0E2AEC05F0E8CF95
:1019C00001F1100E2AEC05F0E8CF02F1110E2AEC1D
:1019D00005F0E8CF03F10101000E046F000E056F62
:1019E000010E066F000E076FFFEC11F06BEC12F0AA
:1019F0001EC182F40401300E822790EC06F01FC154
:101A000082F40401300E822790EC06F020C182F4AB
:101A10000401300E822790EC06F021C182F404010B
:101A2000300E822790EC06F022C182F40401300EC1
:101A3000822790EC06F023C182F40401300E822745
:101A400090EC06F024C182F40401300E822790EC61
:101A500006F025C182F40401300E822790EC06F0D6
:101A600004012E0E826F90EC06F026C182F4040170
:101A7000300E822790EC06F027C182F40401300E6C
:101A8000822790EC06F004016D0E826F90EC06F058
:101A90001200120E2AEC05F0E8CF00F1130E2AEC2A
:101AA00005F0E8CF01F1140E2AEC05F0E8CF02F1C1
:101AB000150E2AEC05F0E8CF03F101010A0E046FC0
:101AC000000E056F000E066F000E076FE0EC11F0C0
:101AD000000E046F120E056F000E066F000E076FEA
:101AE000FFEC11F06BEC12F01EC182F40401300E19
:101AF000822790EC06F01FC182F40401300E822789
:101B000090EC06F020C182F40401300E822790ECA4
:101B100006F021C182F40401300E822790EC06F019
:101B200022C182F40401300E822790EC06F023C11A
:101B300082F40401300E822790EC06F024C182F476
:101B40000401300E822790EC06F004012E0E826F05
:101B500090EC06F025C182F40401300E822790EC4F
:101B600006F026C182F40401300E822790EC06F0C4
:101B700027C182F40401300E822790EC06F00401A4
:101B8000730E826F90EC06F012000A0E2AEC05F03C
:101B9000E8CF00F10B0E2AEC05F0E8CF01F10C0EB6
:101BA0002AEC05F0E8CF02F10D0E2AEC05F0E8CFA3
:101BB00003F1FAEF0DF0060E2AEC05F0E8CF00F184
:101BC000070E2AEC05F0E8CF01F1080E2AEC05F02B
:101BD000E8CF02F1090E2AEC05F0E8CF03F1FAEFA5
:101BE0000DF00101C8EC12F007844AC100F14BC1AD
:101BF00001F107940101E80E046F800E056F000EDD
:101C0000066F000E076FE0EC11F0000E046F040E7B
:101C1000056F000E066F000E076FFFEC11F0880EC7
:101C2000046F130E056F000E066F000E076FD1ECE8
:101C300011F00A0E046F000E056F000E066F000E05
:101C4000076FFFEC11F06BEC12F001011D672EEF36
:101C50000EF00401200E826F31EF0EF004012D0E04
:101C6000826F90EC06F024C182F40401300E8227CA
:101C700090EC06F025C182F40401300E822790EC2E
:101C800006F026C182F40401300E822790EC06F0A3
:101C900004012E0E826F90EC06F027C182F404013D
:101CA000300E822790EC06F00401430E826F90EC18
:101CB00006F0120087C31EF188C31FF189C320F10B
:101CC0008AC321F18BC322F18CC323F18DC324F18C
:101CD0008EC325F190C326F191C327F1010115ECC4
:101CE00013F08DEC12F00101000E046F000E056F71
:101CF000010E066F000E076FE0EC11F00E0E0C6E79
:101D000000C10BF014EC05F00F0E0C6E01C10BF0CE
:101D100014EC05F0100E0C6E02C10BF014EC05F083
:101D2000110E0C6E03C10BF014EC05F004017A0ED9
:101D3000826F90EC06F004012C0E826F90EC06F09E
:101D40000401350E826F90EC06F004012C0E826FB8
:101D500090EC06F0D6EC0CF0D1EF09F087C31EF141
:101D600088C31FF189C320F18AC321F18BC322F1FB
:101D70008CC323F18DC324F18EC325F190C326F1CA
:101D800091C327F1010115EC13F08DEC12F0880ED0
:101D9000046F130E056F000E066F000E076FD5EC73
:101DA00011F0000E046F040E056F000E066F000E9A
:101DB000076FE0EC11F00101E80E046F800E056F73
:101DC000000E066F000E076FFFEC11F00A0E0C6E8E
:101DD00000C10BF014EC05F00B0E0C6E01C10BF002
:101DE00014EC05F00C0E0C6E02C10BF014EC05F0B7
:101DF0000D0E0C6E03C10BF014EC05F004017A0E0D
:101E0000826F90EC06F004012C0E826F90EC06F0CD
:101E10000401360E826F90EC06F004012C0E826FE6
:101E200090EC06F0C5EC0DF0D1EF09F087C31EF180
:101E300088C31FF189C320F18AC321F18BC322F12A
:101E40008CC323F18DC324F18FC325F190C326F1F8
:101E500091C327F1010115EC13F08DEC12F0000E87
:101E6000046F120E056F000E066F000E076FE0EC98
:101E700011F001010A0E046F000E056F000E066FCF
:101E8000000E076FFFEC11F0120E0C6E00C10BF08C
:101E900014EC05F0130E0C6E01C10BF014EC05F000
:101EA000140E0C6E02C10BF014EC05F0150E0C6E46
:101EB00003C10BF014EC05F004017A0E826F90EC74
:101EC00006F004012C0E826F90EC06F00401370E30
:101ED000826F90EC06F004012C0E826F90EC06F0FD
:101EE00049EC0DF0D1EF09F087C31EF188C31FF153
:101EF00089C320F18AC321F18BC322F18CC323F162
:101F00008DC324F18EC325F190C326F191C327F12F
:101F1000010115EC13F08DEC12F0880E046F130E16
:101F2000056F000E066F000E076FD5EC11F0000E66
:101F3000046F040E056F000E066F000E076FE0ECD5
:101F400011F00101E80E046F800E056F000E066FA0
:101F5000000E076FFFEC11F0060E0C6E00C10BF0C7
:101F600014EC05F0070E0C6E01C10BF014EC05F03B
:101F7000080E0C6E02C10BF014EC05F0090E0C6E8D
:101F800003C10BF014EC05F004017A0E826F90ECA3
:101F900006F004012C0E826F90EC06F00401380E5E
:101FA000826F90EC06F004012C0E826F90EC06F02C
:101FB000DBEC0DF0D1EF09F081A89AEF10F007A843
:101FC00053EF10F00101800E006F1A0E016F060E24
:101FD000026F000E036F3EC104F13FC105F140C125
:101FE00006F141C107F1D1EC11F003BF9AEF10F0F7
:101FF000D8EC10F03EC100F13FC101F140C102F147
:1020000041C103F10782DEEC10F00CC104F10DC1F7
:1020100005F10EC106F10FC107F1F80E006FCD0EEC
:10202000016F660E026F030E036FD1EC11F00E0EFE
:102030000C6E00C10BF014EC05F00F0E0C6E01C11C
:102040000BF014EC05F0100E0C6E02C10BF014EC4A
:1020500005F0110E0C6E03C10BF014EC05F00784B3
:102060000101C8EC12F04AC100F14BC101F1079423
:102070000A0E0C6E00C10BF014EC05F00B0E0C6E8A
:1020800001C10BF014EC05F00C0E0C6E02C10BF04C
:1020900014EC05F00D0E0C6E03C10BF014EC05F002
:1020A00007989AEF10F007AA9AEF10F00784010141
:1020B000C8EC12F04AC100F14BC101F10794060EC1
:1020C0000C6E00C10BF014EC05F0070E0C6E01C194
:1020D0000BF014EC05F0080E0C6E02C10BF014ECC2
:1020E00005F0090E0C6E03C10BF014EC05F007842B
:1020F00055C100F156C101F157C102F158C103F1B8
:102100000794120E0C6E00C10BF014EC05F0130EC8
:102110000C6E01C10BF014EC05F0140E0C6E02C134
:102120000BF014EC05F0150E0C6E03C10BF014EC63
:1021300005F0079A0401805181197F0B0BE09EA8DE
:1021400009D014EE00F081517F0BE126E750812B7E
:102150000F01AD6E15EF06F00CC100F10DC101F1DC
:102160000EC102F10FC103F1000E046F000E056FE6
:10217000010E066F000E076FFFEC11F01DA1D7EFE7
:1021800010F01451D8B4D7EF10F00CC100F10DC10C
:1021900001F10EC102F10FC103F1000E046F000E38
:1021A000056F0A0E066F000E076FFFEC11F01200AC
:1021B00001010C6B0D6B0E6B0F6B120001010053D4
:1021C00005E1015303E1025301E1002BA1EC11F001
:1021D000C8EC12F02C51006F2D51016F420E046FAC
:1021E0004B0E056F000E066F000E076FE0EC11F04E
:1021F00000C104F101C105F102C106F103C107F1FB
:102200000CC100F10DC101F10EC102F10FC103F1CA
:1022100007B20FEF11F0D5EC11F011EF11F0D1EC86
:1022200011F000C10CF101C10DF102C10EF103C1A9
:102230000FF11200C8EC12F04CC100F14DC101F1D8
:10224000060E2AEC05F0E8CF04F1070E2AEC05F0A3
:10225000E8CF05F1080E2AEC05F0E8CF06F1090EEB
:102260002AEC05F0E8CF07F1D1EC11F000C118F12C
:1022700001C119F102C11AF103C11BF1290E046F4A
:10228000000E056F000E066F000E076FE0EC11F0F8
:10229000EE0E046F430E056F000E066F000E076F03
:1022A000D5EC11F018C104F119C105F11AC106F1FC
:1022B0001BC107F1E0EC11F000C110F101C111F1F7
:1022C00002C112F103C113F1120E2AEC05F0E8CF9E
:1022D00004F1130E2AEC05F0E8CF05F1140E2AECF8
:1022E00005F0E8CF06F1150E2AEC05F0E8CF07F16E
:1022F0000D0E006F000E016F000E026F000E036FD7
:10230000E0EC11F0180E046F000E056F000E066F62
:10231000000E076FFFEC11F010C104F111C105F1BF
:1023200012C106F113C107F1D5EC11F06A0E046F6A
:102330002A0E056F000E066F000E076FD1EC11F02C
:102340001200BF0EFA6E200E2D6F2C6BD890003746
:10235000013702370337D8B0B2EF11F02D2FA7EFB6
:1023600011F02C072D070353D8B412000331070BCB
:102370008009326F03390F0B010F2C6F80EC5FF077
:10238000336F2C0580EC5FF0335D335F2C6B3233A1
:10239000D8B02C272C3332A9C7EF11F033512C279A
:1023A0001200EDEC12F0D8B0120003510719286F9B
:1023B000B0EC12F0D8900751031928AF800F12002B
:1023C000286BD4EC12F0D8A0EAEC12F0D8B01200CE
:1023D000BFEC12F0C8EC12F01F0E296F00EC13F0E6
:1023E0000B35D8B0B0EC12F0D8A00335D8B012003D
:1023F000292FEEEF11F028B1D7EC12F01200286B64
:1024000004510511061107110008D8A0D4EC12F0F0
:10241000D8A0EAEC12F0D8B01200086B096B0A6B76
:102420000B6B00EC13F01F0E296F00EC13F007513B
:102430000B5DD8A428EF12F006510A5DD8A428EF4E
:1024400012F00551095DD8A428EF12F00451085D7F
:10245000D8A03BEF12F00451085F0551D8A0053D0C
:10246000095F0651D8A0063D0A5F0751D8A0073D75
:102470000B5FD8900081292F15EF12F028B1D7EC0F
:1024800012F0286BD4EC12F0D89004EC13F0075142
:102490000B5DD8A458EF12F006510A5DD8A458EF8E
:1024A00012F00551095DD8A458EF12F00451085DEF
:1024B000D8A067EF12F0003F67EF12F0013F67EF1F
:1024C00012F0023F67EF12F0032BD8B4120028B1CC
:1024D000D7EC12F012000101286BD4EC12F0D8B046
:1024E000120009EC13F0200E296F00370137023774
:1024F000033711EE27F00A0E2A6FE7360A0EE75C63
:10250000D8B0E76EE5522A2F7DEF12F0292F75EF34
:1025100012F028B11D81D890120001010A0E286F17
:10252000200E296F11EE1DF028512A6F0A0ED89047
:10253000E652D8B0E726E7322A2F98EF12F003339D
:10254000023301330033292F92EF12F0E750FF0FCF
:10255000D8A00335D8B012001DB1D7EC12F012008C
:10256000045100270551D8B0053D01270651D8B0C8
:10257000063D02270751D8B0073D0327120000513E
:10258000086F0151096F02510A6F03510B6F12005E
:102590000101006B016B026B036B12000101046B04
:1025A000056B066B076B12000335D8A012000351B0
:1025B000800B001F011F021F031F003FE7EF12F0F7
:1025C000013FE7EF12F0023FE7EF12F0032B282B59
:1025D000032512000735D8A012000751800B041FF5
:1025E000051F061F071F043FFDEF12F0053FFDEF1B
:1025F00012F0063FFDEF12F0072B282B07251200E3
:102600000037013702370337083709370A370B37E6
:1026100012001D6B1E6B1F6B206B216B226B236BDB
:10262000246B256B266B276B12001E510F0B1E6F40
:102630001F510F0B1F6F20510F0B206F21510F0BDC
:10264000216F22510F0B226F23510F0B236F245147
:102650000F0B246F25510F0B256F26510F0B266F83
:0826600027510F0B276F120038
:10BF0000E844F926000C160C2B0C3F0C520C640C68
:10BF1000760C860C960CA50CB30CC10CCF0CDC0C6B
:06BF2000E80CF40C000C1B
:00000001FF
